:0300000002521990
:0C52190078FFE4F6D8FD75817F0252603A
:10249D0020000A3C2E2E2E3E004950436F6E6E6575
:1024AD0063745245510A004950436F6E6E656374F3
:1024BD00000A49504E6F41434B210A003E432C56B2
:1024CD002C43432CC0E4E0EFF2E5F020D1E8EDEA37
:1024DD00EEEC49500A003E432C4D41432C25303241
:1024ED0062583A25303262583A25303262583A25D0
:1024FD00303262583A25303262583A2530326258BD
:10250D002C4D414320E0E4F0E5F10A003E432C560A
:10251D0045522C20332E3220EEF2202573202573C8
:10252D002CC2E5F0F1E8FF20495020ECEEE4F3EB8E
:10253D00FF0A004D617920323320323031320030C4
:10254D00393A33323A3237003E432C4C442C5052F8
:10255D004F473A20202020202020202020202020FE
:10256D00202020202020202020202020202020205E
:10257D00202020202020202020202020202020204E
:10258D00202020202020202020202020202020203E
:10259D0020202020202020202CC4E0F2E020EFF08D
:1025AD00EEF8E8E2EAE828F4E0E9EB290A003E2A31
:1025BD002C312CCEF1EDEEE2EDFBE520EFE0F0E07D
:1025CD00ECE5F2F0FB20F1E5F2E5E2EEE3EE20E8DA
:1025DD00EDF2E5F0F4E5E9F1E00A003E412C413081
:1025ED00312C2562752E2562752E2562752E25627C
:1025FD00752C495020E0E4F0E5F120E0E4E0EFF245
:10260D00E5F0E00A003E412C4130322C2562752E5A
:10261D002562752E2562752E2562752C495020E098
:10262D00E4F0E5F120EEF1ED2E20F1E5F0E2E5F03C
:10263D00E00A003E412C4130332C2562752E256277
:10264D00752E2562752E2562752C495020E0E4F01B
:10265D00E5F120F0E5E72E20F1E5F0E2E5F0E00A06
:10266D00003E412C4130342C2562752E2562752E8D
:10267D002562752E2562752CCCE0F1EAE020F1E59E
:10268D00F2E80A003E412C4130352C2562752E258D
:10269D0062752E2562752E2562752CD8EBFEE70A24
:1026AD00003E2A2C312CC4EEEF2E20EFE0F0E0ECB2
:1026BD00E5F2F0FB20F1E5F2E5E2EEE3EE20E8EDE8
:1026CD00F2E5F0F4E5E9F1E00A003E422C53303139
:1026DD002C2562752CC6E4E0F2FC20E7E0EFF0EE6D
:1026ED00F1E020F1EEE5E4E8EDE5EDE8FF20EEF2B6
:1026FD0020F1E5F0E2E5F0E00A003E422C533032E5
:10270D002C2562752CCEE1ECE5ED20F120F1E5F004
:10271D00E2E5F0EEEC20E1E5E720EAE2E8F2E0EDBB
:10272D00F6E8E90A003E422C5330332C2562752C15
:10273D00CFE5F0E5E7E0EFF3F1EA20EFF0E820EF89
:10274D00EEF2E5F0E520F1E2FFE7E820F120F1E51A
:10275D00F0E2E5F0EEEC0A003E422C5330382C2529
:10276D0062752CCCE5E4EBE5EDEDFBE9204950205D
:10277D00EAE0EDE0EB28E7E0E4E5F0E6EAE020E46E
:10278D00EE203520F1E5EA290A003E422C53303582
:10279D002C2562752CCAE0EDE0EB20F8E8F0EEEAAE
:1027AD00EEE2E5F8E0F2E5EBFCEDEEE3EE20EEE136
:1027BD00ECE5EDE00A003E532C5330362C2530323B
:1027CD0062582530326258253032625825303262D7
:1027DD0058253032625825303262582C4D414320F5
:1027ED00E0E4F0E5F120F8E8F0EEEAEEE2E5F8E0FD
:1027FD00F2E5EBFCEDEEE3EE20EEE1ECE5EDE00ACB
:10280D00003E454E440A000A44756D705820202044
:10281D002020303020303120303220303320303401
:10282D0020303520303620303720303820303920D8
:10283D00304120304220304320304420304520307C
:10284D0046000A3A003A20000A000A44756D7044A9
:10285D0020202020203030203031203032203033E5
:10286D00203034203035203036203037203038209D
:10287D003039203041203042203043203044203048
:10288D004520304600457272206B657900526420F8
:10289D00656570726F6D0A005264204D454D0A00DA
:1028AD00526420436F64650A005772697465204352
:1028BD006F64650A0044656275674950204F4E0A82
:1028CD000044656275674950204F46460A004465CD
:1028DD0062756755736572204F6E0A0044656275A7
:1028ED006755736572204F46460A004465627567E9
:1028FD004D7367204F6E0A0044656275674D7367AF
:10290D00204F46460A00436F6E666967206C6F6301
:10291D006B210A00577220656570726F6D0A002079
:10292D005361766520656570726F6D210A00457281
:10293D0072204D414321004C6F61643E3E002A00E0
:10294D00CEF8E8E1EAE00A00202D2025752825754E
:10295D00290A003C4130313D003C4130323D003CC4
:10296D004130333D003C4130343D003C4130353D3C
:10297D00003C21003C5330313D003C5330323D0092
:10298D003C5330333D003C5330353D003C533038E3
:08299D003D003C5330363D00C3
:065C0B000113000111006D
:105DA800C28E438910E4F58B758DB8D2ABD28E22A2
:03001B000250FA96
:1050FA00C0E0C083C082C0D0C28E758B00758DB8E7
:10510A0020280675A61E75A6E10511D224E51360AE
:10511A000205130516E516540F7051E512D39401D2
:10512A0040021512D230E516543F7012D222907FF7
:10513A0069E0600A04F0E0D394B44002D228907F78
:10514A0062E0600204F09079DFE0600214F0907F80
:10515A006AE0D394014003E014F03027020514E515
:10516A0015D394644004D22880020515E510D3941F
:10517A000140021510D28ED0D0D082D083D0E03236
:101E2400C291C290D2B5C22D7D027C007F07125DA3
:101E3400028F28E528646060097D017F60125C7D63
:101E4400D22DE4FDFC7F0B125D028F28E52830E6DD
:101E5400097D04E4FF125CA1D22D7D017C007F0783
:101E6400125D028F28E5287008FD7FFF125C7DD289
:101E74002D302D03126000C288C2A8C2AA75890041
:101E8400125527907C1AE0B4FA06A3E064CE607B76
:101E9400E4F52874122528F582E4347CF583E4F013
:101EA4000528E528B443EC907C1A74FAF0A374CEA8
:101EB400F0A374CCF0907C20740AF0E4A3F0A304A3
:101EC400F0A3F0907C1674FFF0A3F0A3F0E4A3F069
:101ED400907C317403F0E4F528E5282401FFE43311
:101EE400FE74122528F582E4347CF583E0FD125C4F
:101EF400590528E528C3944340DFE4F5A775A61ED9
:101F040075A6E1907FF0F0A3F080FE907C25740329
:101F1400F0A374CCF0E4907C24F0907F67F0A3F0FD
:101F2400124ABCC2B5124F9EC228125812D22DC2F8
:101F34002FC22E907E527408F0907B907424F0E4AB
:101F4400A3F0907C1AE0907B92F0907C1BE0907B55
:101F540093F0907C1CE0907B94F0907C1DE0907B4F
:101F640095F0907C1EE0907B96F0907C1FE0907B37
:101F740097F0751201E4907E53F0C229C22AC22B55
:101F8400C22C202D18AF28FE7D03124BA2E4FF12B1
:101F940050517E247F9DE4FBFDFC1249BC907F6977
:101FA400E060037401F0E49079DFF0F514907E5161
:101FB400F0F515125DA875A70775A61E75A6E1D2E2
:101FC400AFE4F5159079DFE0700312108C907F6A0E
:101FD400E06401701D9080007410F09080A874FF7C
:101FE400F0A3F0A3F0A3F0E4907F6AF0D22DC22E08
:101FF400C22F908008E0F52830E405D2297410F04F
:10200400E52830E508D22B9080087420F0E52830CC
:10201400E608D22A9080087440F0E514C394034083
:1020240019908002E4F0908001F0908000F0E514B3
:1020340094064006E4F5141258129080A0E0700350
:1020440012561F9080B8E070031255A59080D0E01E
:1020540070031257B6908000E070133029101248B4
:10206400B8907C0DEFF0D3940040031200369080BA
:1020740002E07006908000E06005D227021FC5C20E
:1020840027E4F5149079DFE06003021FC5202D12C8
:10209400907E54E0600C7E247F9F124D50E4907E2D
:1020A40054F0302B12124296907C0DEFF0D3940032
:1020B4004005E0FF121761202A03022249123F91D2
:1020C400907C0DEFF07003021FC5907C51E054BF6B
:1020D400247F70030221A414700302217C24026073
:1020E400030221EB202D077E247FA6124D502031C0
:1020F40003022249907C29E07006907C2DE0606701
:10210400907F5EE0FF907C29E0B50724907F5FE03C
:10211400FE907C2AE0B50618907F60E0FE907C2B50
:10212400E0B5060C907F61E0FE907C2CE06E603799
:10213400907C2DE06F6003022249907F5FE0FF9066
:102144007C2EE06F6003022249907F60E0FF907C68
:102154002FE06F6003022249907F61E0FF907C30A2
:10216400E06F6003022249C225907E537401F0128D
:102174005DCF751201022249907F69E0600374010A
:10218400F0907F56E0FF907C53E06F600302224999
:10219400907F56E004F0E4F512907E51F00222495B
:1021A400302503022249907C20E07003021FC59071
:1021B4007B8FE06008907C31741EF08006907C3147
:1021C4007403F0125DCED225E4F512907E51F090A6
:1021D4007F6204F0E4907F55F0A3F0202D677E2405
:1021E4007FB4124D50805E907F69E060037401F00B
:1021F400302552907C51E020E74B907C53E0FF90D7
:102204007F55E0FE6F600D907F5DE07007EE146F08
:1022140070338013907F55E004F0907C0DE0FFD381
:10222400940440031200329078DB7482F0A37401AA
:10223400F0907C53E09078DDF07E787FDB7D0312B4
:102244005429021FC520250302236CE512706E1267
:102254005BA9EF60237E7D7F51907D52E02404FDD5
:10226400125429907F5DE07009907C31E0F51202F0
:102274001FC5E4F512021FC5907F62E0D3943C4071
:102284003C907F5DE07036907B8FE07030907F6291
:1022940004F0124EE9E4907D51F0A37412F0907FA3
:1022A40056E0907D53F0A374FDF09079E063A201B1
:1022B400907D5563A2017F12123CDF8098125DC3AA
:1022C4008F28E528B401159078DB7483F0E4A3F03B
:1022D4007E787FDB7D02125429021FC5E528D39442
:1022E40001401C9078DB7483F0A37401F0E528248A
:1022F400FEA3F07E787FDB7D03125429021FC5E51F
:102304001264016003021FC5907E51E004F0202D89
:10231400077E247FBE124D50907E51E0FFD394017E
:10232400400B907C31E0941E5003E004F0EFC39422
:1023340005400DC225E4907E53F0125DCF021FC507
:102344007C7F7D5E907C25E0FAA3E0FB7F02125245
:10235400A57E7D7F51907D52E02404FD1254299086
:102364007C31E0F512021FC5E51264016003021F0F
:10237400C5907E53E014604624FE6042147003024C
:10238400245F24046003021FC5E4F5142031139074
:102394007E537404F0907E51E05401F075120102F2
:1023A4001FC59080027410F0E4907E53F0907E512B
:1023B40004F0751212907F5E74FFF0021FC5907FC7
:1023C4005EE07003022449907D517480F0907D5347
:1023D4007401F0E4A3F0A304F0A37430F0A3747BBD
:1023E400F0E4F52874582528F582E4347DF58374E7
:1023F4007DF074592528F582E4347DF583E4F0E515
:10240400282407907D52F07C7F7D5E907C25E0FA45
:10241400A3E0FB7F021252A57E7D7F51E5282409AB
:10242400FD125429907F5DE0601B125DCED225E43D
:10243400F512907E51F0907F6204F0E4907F55F0A5
:10244400A3F0021FC5303107E4907E53F08006905C
:102454007E537404F0751212021FC590800274102A
:10246400F0751203907E51E06401FFF0907E537486
:1024740001F0EF7012907C2DE0600C122CB8907F6C
:102484005E122CD0021FC5907C29122CB8907F5E5E
:08249400122CD0021FC580FECE
:01249C00221D
:10003600907C52E0B444047F0180027F00907C51A2
:10004600E0B447047E0180027E00EE5F604A907C49
:100056001AE0907C53F0907C1BE0907C54F0907CEE
:100066001CE0907C55F0907C1DE0907C56F0907CD6
:100076001EE0907C57F0907C1FE0907C58F0907CBE
:10008600527452F0907B8963A2019080A863A2010A
:100096007F06123CDF020913907C0DE0C3940850E2
:1000A6000302091C907C1AE0FF907C53E06F60030A
:1000B60002091C907C1BE0FF907C54E06F600302F9
:1000C600091C907C1CE0FF907C55E06F60030209E0
:1000D6001C907C1DE0FF907C56E06F600302091CBB
:1000E600907C1EE0FF907C57E06F600302091C9035
:1000F6007C1FE0FF907C58E06F600302091C907C37
:1001060052E06444701A9080A8E0B4FF13907B8993
:1001160063A2019080A863A2017F06123CDF8010D3
:10012600907B8DE09080ACF0907B8EE09080ADF07F
:10013600907F69E060037401F0907F6A7464F090C8
:100146007C527452F0907C51E0646D60030202BAF6
:100156007BFF7A2479C91231BB7BFF7A2479E3903D
:100166007C1AE0F535A3E0F536A3E0F537A3E0F514
:1001760038A3E0F539A3E0F53A1231BB7535FF75C2
:1001860036257537407538FF753925753A4C7BFF2E
:100196007A2579191231BB7BFF7A2579551231BB45
:1001A6007BFF7A2579BB1231BB7BFF7A2579E890F4
:1001B6007C20E0F535A3E0F536A3E0F537A3E0F5BE
:1001C600381231BB7BFF7A267912907C29E0F5350F
:1001D600A3E0F536A3E0F537A3E0F5381231BB7B93
:1001E600FF7A267940907C2DE0F535A3E0F536A31D
:1001F600E0F537A3E0F5381231BB7BFF7A26796E3E
:10020600907C16E0F535A3E0F536A3E0F537A3E0DC
:10021600F5381231BB7BFF7A267991907C12E0F596
:1002260035A3E0F536A3E0F537A3E0F5381231BB88
:100236007BFF7A2679AE1231BB7BFF7A2679D7A26D
:1002460031E433F5351231BB7BFF7A277907907F8E
:100256005DE0F5351231BB7BFF7A277932907F69F5
:10026600E0F5351231BB7BFF7A277965907B8FE00D
:10027600F5351231BB7BFF7A277997A223E433F554
:10028600351231BB7BFF7A2779C3907F57E0F5356E
:10029600A3E0F536A3E0F537A3E0F538A3E0F5399A
:1002A600A3E0F53A1231BB1239F67BFF7A28790EB4
:1002B6001231BB22907C51E0644C70737E287F140F
:1002C600FBFDFC1249BC907C59E0F529A3E0F52A18
:1002D600E4F52CE529907C5BF0A3E52AF07E287FE7
:1002E6004F7C7C7D5B7B021249BCE4F52B852A8220
:1002F600852983E0FF745B252BF582E4347CF58346
:10030600EFF0052AE52A70020529052BE52BB41026
:10031600DC7E287F527C7C7D5B7B101249BC052CE1
:10032600E52CC3941040AC7E287F55124D50229088
:100336007C51E0646C7060F52D7E287F57FBFDFCD8
:100346001249BCE4F52CE4907C5BF0A3E52DF07E2D
:10035600287F4F7C7C7D5B7B021249BCE4F52BA891
:100366002DE6FF745B252BF582E4347CF583EFF0F4
:10037600052D052BE52BB410E67E287F527C7C7D6F
:100386005B7B101249BC052CE52CC3940840B77E54
:10039600287F55124D5022907C51E0644B7061F5D8
:1003A6002B7443252BF582E4347CF583E0603274AC
:1003B60043252BF582E4347CF583E0F46023744313
:1003C600252BF582E4347CF583E0FF7459252BF563
:1003D60082E4347CF583E0B50710052BE52BB408E1
:1003E600C09079DF7432F0020913907C517421F0C9
:1003F600302D030209137E287F92124D50020913F5
:10040600907C51E0B4521A202D077E287F9A124D17
:1004160050907C517472F07E7C7F517D081253A9F6
:1004260022907C51E064497045202D077E287FA5E7
:10043600124D50907C59E0F529A3E0F52AE4F52BFE
:10044600852A82852983E0FF745B252BF582E434B7
:100456007CF583EFF0052AE52A70020529052BE5D0
:100466002BB480DC7E7C7F517D8A1253A922907C3E
:1004760051E064437046202D077E287FAD124D5013
:10048600907C59E0F529A3E0F52AE4F52B852A822C
:10049600852983E493FF745B252BF582E4347CF590
:1004A60083EFF0052AE52A70020529052BE52BB412
:1004B60080DB7E7C7F517D8A1253A922907C51E09D
:1004C600645A7053202D077E287FB6124D50907CBB
:1004D60059E0F529A3E0F52A7C7C7D5B7B80AF2A79
:1004E600AE29125B75E4F52B852A82852983E49370
:1004F600FF745B252BF582E4347CF583EFF0052A47
:10050600E52A70020529052BE52BB480DB7E7C7F6E
:10051600517D8A1253A922907C51E0644460030203
:1005260005AE907C59E0FF64447003020913EFB4F2
:10053600310CC22D7E287FC2124D50020913907CC9
:1005460059E0B4300CD22D7E287FCE124D500209D0
:1005560013907C59E0B4320CD22E7E287FDB124DEC
:1005660050020913907C59E0B4330CC22E7E287FCA
:10057600E9124D50020913907C59E0B4340CD22F85
:100586007E287FF8124D50020913907C59E0B4354D
:100596000CC22F7E297F05124D50020913907C59FB
:1005A600E0FF125D820209139079DFE07013202DBF
:1005B600077E297F13124D50907C517421F0020959
:1005C600139079DF7432F0907C51E0FFB45104C28D
:1005D600AF80FEEF64577045202D077E297F2112DC
:1005E6004D50907C5AE0907C0DF0E4F52B907C0DFC
:1005F600E0FFE52BC39F4003020913745B252BF52F
:1006060082E4347CF583E0FF907C59E0252B248836
:10061600F582E4347AF583EFF0052B80D0907C5197
:10062600E0645360030206D1202D077E297F2C1239
:100636004D50907C1AE0FF907A91E06F703C907C70
:100646001BE0FF907A92E06F7030907C1CE0FF9088
:100656007A93E0B50724907C1DE0FF907A94E0B58C
:100666000718907C1EE0FF907A95E0B5070C907C09
:100676001FE0FF907A96E06F6016907C517421F02F
:10068600302D030209137E297F3B124D50020913B8
:10069600E4F52BE4F515AF2BFE7488252BF582E4E3
:1006A600347AF583E0FD125C59052BE52BC394FEE5
:1006B60040E1C2AFE4907FF0F0A3F0907FFD74AA12
:1006C600F0A374FFF0A37455F080FE907C51E064B3
:1006D6004F7056907C59E0F529A3E0F52AE52A45A6
:1006E60029700A202D077E297F44124D50202D07A0
:1006F6007E297F4B124D50E4F52B745B252BF5823A
:10070600E4347CF583E0852A82852983F0052AE591
:100716002A70020529052BE52BB480DE907F67E45D
:1007260075F080122AAA020913907C51E064457084
:1007360074907C59E0FEA3E0FF907FF0EEF0A3EF0B
:10074600F0D39400EE94044038907FF0E0FEA3E0EE
:10075600FF907F67E0FCA3E0FD9FEC9E4023E42F23
:10076600FFEE3401FED3ED9FEC9E5015C2AF907F95
:10077600FD74AAF0A374FFF0A37455F0E4F5A78006
:10078600FE7E297F4D124D507BFF7A297955907F49
:10079600F0E0F535A3E0F536907F67E0F537A3E0A6
:1007A600F5381231BB907C51E06465600302091C88
:1007B600907C59E0FFA3E0907FF0CFF0A3EFF0E448
:1007C600F529F52AD3907FF1E0952A907FF0E09500
:1007D600294020E4F515252AFFE5293401FE852A5E
:1007E60082852983E0FD125C59052AE52A700205F7
:1007F6002980D17E297F60125329EF4E6020120096
:1008060003907C20EFF0120003907C21EFF01200A1
:1008160003907C22EFF0120003907C23EFF07E29F8
:100826007F66125329EF4E6020120003907C29EF59
:10083600F0120003907C2AEFF0120003907C2BEF5D
:10084600F0120003907C2CEFF07E297F6C12532966
:10085600EF4E6020120003907C2DEFF01200039003
:100866007C2EEFF0120003907C2FEFF01200039025
:100876007C30EFF07E297F72125329EF4E602012F2
:100886000003907C16EFF0120003907C17EFF01235
:100896000003907C18EFF0120003907C19EFF07EB5
:1008A600297F78125329EF4E6020120003907C12A4
:1008B600EFF0120003907C13EFF0120003907C140B
:1008C600EFF0120003907C15EFF0E4F52BE4F5153C
:1008D600E52B2401FFE433FE7412252BF582E43464
:1008E6007CF583E0FD125C59052BE52BC394434050
:1008F600DCC2AFE4907FF0F0A3F0907FFD74AAF025
:10090600A374FFF0A37455F0E4F5A780FE7E7C7F08
:06091600517D081253A9F7
:01091C0022B8
:105B0500AE07EEC39430400BEED394395005EE2426
:105B1500D0FF22EEC39461400BEED394665005EEA0
:105B250024A9FF22EEC39441400BEED394465005C1
:085B3500EE24C9FF22AF062295
:105D5600907B87E475F001122AAA907B87E0FEA368
:065D6600E0FF125CE522E3
:10000300125D56125B05EFC454F0FEC006125D5636
:08001300125B05D0E02FFF2273
:10575900E4907F72F0125D56907F73EFF0C394303E
:105769004018E0FFD394395011907F72E024E0F59E
:1057790082E43479F583EFF08011907F72E024E0C0
:10578900F582E43479F583E4F0800C907F72E004CB
:10579900F0E0D3940840BE753100753200753300CE
:0C57A900E4F5347B017A7979E0123DEDE3
:0157B50022D1
:045329008E2E8F2F06
:10532D00907B87E4F0A374FFF0125D56EF6069F493
:10533D006066852F82852E83E493B507EC75300169
:10534D00E52F2530F582E4352EF583E49360259025
:10535D007B88E02530FF907B87E03400FE125CE512
:10536D00E52F2530F582E4352EF583E493B507045A
:10537D00053080CCE52F2530F582E4352EF583E41C
:10538D009370A6E53024FFFFE434FF907B878FF008
:0B539D00122AAA7E007F0122E4FEFF1E
:0153A80022E2
:104ABC007E297F7E125329EF4E70037F01227E29BF
:104ACC007F81125329EF4E600C125D56EF24D024D7
:104ADC00FF92318002D2317E297F87125329EF4E0B
:104AEC00600C125D56EF24D0907F5DF08005E49051
:104AFC007F5DF07E297F8D125329EF4E600C125D85
:104B0C0056EF24D0907F69F08005E4907F69F07EA9
:104B1C00297F93125329EF4E600C125D56EF24D06F
:104B2C0024FF92238002C2237E297F99125329EFFE
:104B3C004E600C125D56EF24D0907B8FF08005E414
:104B4C00907B8FF0907C1A63A201907F5763A20137
:104B5C007F06123CDF30233B7E297F9F125329EFC7
:104B6C004E6030120003907F57EFF0120003907FDD
:104B7C0058EFF0120003907F59EFF0120003907F72
:104B8C005AEFF0120003907F5BEFF0120003907F5E
:064B9C005CEFF07F002237
:1059B900907E52E0C3947C40027F0A907E52E0FEC2
:1059C90004F074902EF582E4347BF583EFF0BF0A7E
:1059D90027907E52E0FF04F074902FF582E4347B27
:1059E900F583E4F0907E52E0FF1254A9907E527440
:0959F90008F0907B91E004F0221B
:105812009080007480F0907C1263A201F583F5827F
:1058220063A2017F08123CDF907C1A63A201908080
:105832008863A2017F0A123CDF9080927407F0A372
:1058420074D0F0A37406F0907C24E0FF9080B1F055
:105852009080E1EFF09080957455F0A3F090800075
:0A5862007401F090800974F0F02248
:10561F00908009E04410F09080A0E070609080A12D
:10562F007482F09080A874FFF0A3F0A3F0A3F07F32
:10563F00039080AEEFF0A374CBF09080007402F073
:10564F00907FD3122CDC00000000907FD3E090807D
:10565F0040F0907FD4E0908041F0907FD5E0908033
:10566F0042F0907FD6E0908043F0A3E4F0A3F0A344
:0D567F00F0A3F0908018F0A3F0A3F0A3F0CA
:01568C0022FB
:1057B600908009E04440F09080D17482F07F03909D
:1057C60080DEEFF0A374CCF09080027402F0907F3C
:1057D600D7122CDC00000000907FD7E0908058F0B4
:1057E600907FD8E0908059F0907FD9E090805AF071
:1057F600907FDAE090805BF0A3E4F0A3F0A3F0A33F
:0B580600F0908030F0A3F0A3F0A3F0BE
:015811002274
:1055A500908009E04420F09080B8E0706C9080B95C
:1055B5007482F07F039080C6EFF07FCDA3EFF07F7C
:1055C500039080C4EFF0A374CDF09080C074FFF019
:1055D500A3F0A3F0A3F09080017402F0907FDB129A
:1055E5002CDC00000000907FDBE090804CF0907F89
:1055F500DCE090804DF0907FDDE090804EF0907F74
:10560500DEE090804FF0A3E4F0A3F0A3F0A3F090C8
:095615008024F0A3F0A3F0A3F03F
:01561E002269
:1052A5008C298D2AA907EAFDE975F018A424ACFF1D
:1052B500E5F034808F82F583EDF0EBFDE975F018AC
:1052C500A4FFAEF024ACFBEE34808B82F583A3ED16
:1052D500F0852A828C83E0FDEF24A8FFEE3480FE62
:1052E5008F82F583EDF0852A828C83A3E08F828EF1
:1052F50083A3F0852A82852983A3A3E0FDE975F0C0
:1053050018A424A8FFE5F03480FE8F82F583A3A3BB
:10531500EDF0852A828C83A3A3A3E08F828E83A3DD
:04532500A3A3F0222C
:0653A9008D2EAB07AA06E1
:1053AF00908000E030E507907E547401F022907FEA
:1053BF00D3122CB88F328E318D308C2FAE02AF03BB
:1053CF008E838F8263A201E531540744C0F5838534
:1053DF00328263A201AF2E123D51E4FCFDFEE53295
:1053EF00252EF532EE3531F531ED3530F530EC3522
:1053FF002FF52F908040E52FF0A3E530F0A3E53196
:10540F00F0A3E532F09080007420F0AF32AE31ADF2
:09541F0030AC2F907FD3122CD089
:015428002261
:065429008D29AB07AA0665
:10542F00908002E030E507907E547403F022907F65
:10543F00D7122CB88F2D8E2C8D2B8C2AAE02AF034A
:10544F008E838F8263A201E52C540744D0F58385A8
:10545F002D8263A201AF29123D51E4FCFDFEE52D23
:10546F002529F52DEE352CF52CED352BF52BEC35BF
:10547F002AF52A908058E52AF0A3E52BF0A3E52C16
:10548F00F0A3E52DF09080027420F0AF2DAE2CAD7F
:09549F002BAC2A907FD7122CD00F
:0154A80022E1
:025051008F2F9F
:10505300908001E030E509907E547402F07F0022D5
:10506300907FDB122CB88F338E328D318C30907F52
:105073005763A201E532540744C8F583853382633D
:10508300A2017F06123D67E5332406F533E435328A
:10509300F532E43531F531E43530F530907E556342
:1050A300A201E532540744C8F58385338263A20124
:1050B300AF2F123D67E4FCFDFEE533252FF533EEFC
:1050C3003532F532ED3531F531EC3530F530908050
:1050D3004CE530F0A3E531F0A3E532F0A3E533F07E
:1050E3009080017420F0AF33AE32AD31AC30907F9D
:0650F300DB122CD0AF2FF0
:0150F9002294
:1048B8009081E0E0F529052905290529052905291B
:1048C80005290529052905290529908010E0F52CD9
:1048D800A3E0F52DA3E0F52EA3E0F52F9081E1E00C
:1048E800F529052905290529052905290529052960
:1048F800052905290529908014E0F530A3E0F53154
:10490800A3E0F532A3E0F533E532B52E08E533B57B
:104918002F037F0022E4F529E532540744E0F583AC
:1049280085338263A201907C5163A2017F08123D06
:1049380097907C5363A201907B8963A2017F061242
:104948003CDF907C51E0F52AA3E0F52BE4F52990B3
:104958007C51E0702AA3E024F8F529E53254074495
:10496800E0F58385338274082582F582E43583F582
:104978008363A201907C5163A201AF29123D97AED7
:104988002AE4FCFDE533252BF533E5323EF532ED1F
:104998003531F531EC3530F530908014E530F0A341
:1049A800E531F0A3E532F0A3E533F09080007440E0
:0349B800F0AF2934
:0149BB0022D9
:103F91009081E6E0F5290529052905290529052945
:103FA10005290529052905290529908028E0F52CF1
:103FB100A3E0F52DA3E0F52EA3E0F52F9081E7E036
:103FC100F529052905290529052905290529052990
:103FD10005290529052990802CE0F530A3E0F5316C
:103FE100A3E0F532A3E0F533E4F529E532B52E0A75
:103FF100E533B52F05C22A0240FDE532540744F0EE
:10400100F58385338263A201907C5163A2017F080D
:10401100123D97907C51E0F52AA3E0F52BE52B4565
:104021002A70099080027410F07F0022907F5EE078
:10403100FFF46030907C53E06F60030240C4907FD6
:104041005FE0FF907C54E06F7079907F60E0FF90BB
:104051007C55E06F706D907F61E0FF907C56E06F62
:104061006031805F907C53E0907F5EF0907C54E003
:10407100907F5FF0907C55E0907F60F0907C56E0FF
:10408100907F61F0907C57E0FFA3E0907C25CFF01A
:10409100A3EFF0907C51E0702AA3E024F8F529E524
:1040A10032540744F0F58385338274082582F58202
:1040B100E43583F58363A201907C5163A201AF29AA
:1040C100123D97AE2AE4FCFDE533252BF533E532AD
:1040D1003EF532ED3531F531EC3530F530AF2FAEFF
:1040E1002EAD2DAC2CAB33AA32A931A830D3122C72
:1040F100A740099080027410F07F002290802CE587
:1041010030F0A3E531F0A3E532F0A3E533F0908080
:06411100027440F0AF292A
:014117002285
:104296009081E3E0F5290529052905290529052940
:1042A6000529052905290529052990801CE0F52CF5
:1042B600A3E0F52DA3E0F52EA3E0F52F9081E4E031
:1042C600F529052905290529052905290529052988
:1042D600052905290529908020E0F530A3E0F53170
:1042E600A3E0F532A3E0F533E4F529E532B52E0A6D
:1042F600E533B52F05C22B0243ECE532540744E8FB
:10430600F58385338263A2019078DF63A2017F0E75
:10431600123DAD9078DFE0F52AA3E0F52B9078E723
:10432600E0FFF4604A907F57E0FEEF6E7079A3E0FD
:10433600FF9078E8E06F706F907F59E0FF9078E922
:10434600E06F7063907F5AE0FF9078EAE06F7057F5
:10435600907F5BE0FF9078EBE06F704B907F5CE0C6
:10436600FF9078ECE06F703FE49078EEF080089074
:1043760078EE74FFF0D2D99078DFE0702AA3E024BB
:10438600F2F529E532540744E8F583853382740E45
:104396002582F582E43583F58363A2019078DF6395
:1043A600A201AF29123DADAE2AE4FCFDE533252B73
:1043B600F533E5323EF532ED3531F531EC3530F594
:1043C60030AF2FAE2EAD2DAC2CAB33AA32A931A80F
:1043D60030D3122CA75006E52B452A700990800190
:1043E6007410F07F0022908020E530F0A3E531F0D4
:1043F600A3E532F0A3E533F09080017440F0AF29D5
:014406002293
:044D50008E2E8F2FE5
:104D5400908000E030E507907E547401F022907F4B
:104D6400D3122CB88F358E348D338C32E535FFE574
:104D7400345407FEE42FF531EE34C0F5308531822A
:104D8400F5837423F00531E531700205305330C7E3
:104D9400F582853083740AF00531E53170020530FF
:104DA4005330C7907C1A63A20185308385318263B6
:104DB400A2017F06123D5174062531F531E43530E8
:104DC400F530852E83852F8263A20185308385315A
:104DD4008263A201123D35E4FCFDFE907FD3122CC8
:104DE400C4122B6FEF2408FFE43EFEE43DFDE43CD7
:104DF400FC907FD3122CD0907FD3E0908040F09031
:104E04007FD4E0908041F0907FD5E0908042F09094
:0D4E14007FD6E0908043F09080007420F085
:014E2100226E
:0A49BC008E358F368C378D388B391D
:1049C600908000E030E507907E547401F022907FDD
:1049D600D3122CB88F3F8E3E8D3D8C3CE53FFFE5D4
:1049E6003E5407FEE42FF53BEE34C0F53A853B8294
:1049F600F5837423F0053BE53B7002053A533AC74D
:104A0600F582853A83740AF0053BE53B7002053A68
:104A1600533AC7907C1A63A201853A83853B826329
:104A2600A2017F06123D517406253BF53BE4353A5B
:104A3600F53A85358385368263A201853A83853BBF
:104A46008263A201123D358F40EF253BF53BE435ED
:104A56003AF53AE539601785378385388263A201CE
:104A6600853A83853B8263A201AF39123D51E54009
:104A760024082539F539FFE4FCFDFEE53F2FF53F17
:104A8600EE353EF53EED353DF53DEC353CF53C90DD
:104A96008040E53CF0A3E53DF0A3E53EF0A3E53F0D
:104AA600F09080007420F0AF3FAE3EAD3DAC3C9040
:054AB6007FD3122CD09B
:014ABB0022D8
:064C7C008E2E8F2F8D30FB
:104C8200908000E030E507907E547401F022907F1E
:104C9200D3122CB88F368E358D348C33E536FFE542
:104CA200355407FEE42FF532EE34C0F531853282F9
:104CB200F5837423F00532E532700205315331C7B2
:104CC200F582853183EBF00532E53270020531530E
:104CD20031C7907C1A63A20185318385328263A237
:104CE200017F06123D5174062532F532E43531F565
:104CF20031852E83852F8263A2018531838532829D
:104D020063A201AF30123D5174082530F530FFE443
:104D1200FCFDFEE5362FF536EE3535F535ED35344D
:104D2200F534EC3533F533908040E533F0A3E534C8
:104D3200F0A3E535F0A3E536F09080007420F0AFE3
:0D4D420036AE35AD34AC33907FD3122CD09B
:014D4F002241
:0254A9008F462C
:1054AB00908000E030E507907E547401F022907FED
:1054BB00D3122CB88F4A8E498D488C47E54AFFE5AD
:1054CB00495407FEE42FFFEE34C0907B9063A2019A
:1054DB00F5838F8263A201AF46123D51E4FCFDFEC2
:1054EB00E54A2546F54AEE3549F549ED3548F54887
:1054FB00EC3547F547908040E547F0A3E548F0A32E
:10550B00E549F0A3E54AF09080007420F0AF4AAE75
:0B551B0049AD48AC47907FD3122CD064
:015526002262
:064BA2008E298F2AAB05ED
:104BA800908000E030E507907E547401F022907FF9
:104BB800D3122CB88F308E2F8D2E8C2DE530FFE53B
:104BC8002F5407FEE42FF52CEE34C0F52B852C82EC
:104BD800F5837423F0052CE52C7002052B532BC7A5
:104BE800F582852B83EBF0052CE52C7002052B90C4
:104BF8007C1A63A201852B83852C8263A2017F0620
:104C0800123D517406252CF52CE4352BF52B532B2E
:104C1800C7E529852C82852B83F0052CE52C7002AD
:104C2800052B532BC7F582852B83E52AF0052CE548
:104C38002C7002052B532BC7E530240AF530E435D8
:104C48002FF52FE4352EF52EE4352DF52D908040E7
:104C5800E52DF0A3E52EF0A3E52FF0A3E530F090C5
:104C680080007420F0AF30AE2FAD2EAC2D907FD3E6
:034C7800122CD02B
:014C7B002216
:0A5DB800E4FEEEC39F50030E80F8D6
:015DC20022BE
:105CE500A2AF9232C2AF438E2075D2028F828E83CD
:0C5CF500E0FFE4F5D2538EDFA23292AF44
:015D0100227F
:105C5900E5D220E0FBA2AF9232C2AF43D2028F82DB
:105C69008E83EDF075D25063D250A23292AFE5D255
:035C790020E0FB2D
:015C7C002205
:10552700E4FDED2401FFE433FE125CE574122DF572
:1055370082E4347CF583EFF00DBD3FE6E4FDED2416
:105547007FFFE433FE125CE574082DF582E4347ABC
:10555700F583EFF074082DF582E4347AF583E07073
:105567001B74082DF582E4347AF5837420F07409EE
:105577002DF582E4347AF583E4F080040DBD80BE16
:10558700E4907A87F0FDEDFF7E00125CE574882DCC
:0D559700F582E4347AF583EFF00DBDFEE9F6
:0155A40022E4
:025B75008B2E75
:105B7700A2AF9232C2AF85A22F53A2FE8E838F822D
:105B870005A28C838D827409123DDBE52E53A2FE9C
:105B970043A220123DDD53A2DF852FA2A23292AF8E
:015BA700FFFE
:015BA80022DA
:105D0200A2AF9232C2AF8C838D82EF123DDB43A2EF
:0C5D120020123DDD53A2DFA23292AFFF51
:015D1E002262
:025C7D008F296D
:105C7F00A2AF9232C2AFE4F5838D827406123DDB80
:105C8F00E52943A220123DDD53A2DFA23292AF7F5E
:015C9F000103
:015CA00022E1
:025CA1008F2949
:105CA300A2AF9232C2AFE4F5838D82740A123DDB58
:105CB300E52943A220123DDD53A2DFA23292AF7F3A
:015CC30001DF
:015CC40022BD
:103C0400A907E7FFA805EF93C3966008403B74FC3F
:103C14002FFF80F00F08EF93C3966008402B74FBCE
:103C24002FFF80E00F08EF93C3966008401B74FADF
:103C34002FFF80D00F08EF93D3966008400B74F9E0
:103C44002FFF80C01F1F1F1F1FEF54FEF80303F731
:103C5400E893FC08E893FD08E893FE08E893FF2244
:103C640009E993C39D6008402974FB29F980F1098F
:103C7400E993C39E6008401A74FA29F980E209E9BD
:103C840093D39F6008400B74F929F980D31919194B
:103C94001919E9C313C313FF22740093F8ECC398F2
:103CA4004024701F740193F8EDC398401970147484
:0E3CB4000293F8EEC398400E7009740393F863
:103CC200EFC39840037F00227F0122EDF8E6F0085F
:103CD200A3DFFA22EDF8E0F608A3DFFA22E0A363FD
:103CE200A201F0A363A201DFF475A2002263A20184
:103CF200F0A363A20122E0A363A201F0A363A201E5
:103D0200E0A363A201F0A363A201E463A201F0A312
:103D120063A201DFE175A20022E0A363A2016DFEAE
:103D2200936CFDEE058393FC158363A201DFEA75B4
:103D3200A200227F00E493A363A201F00F600CA310
:103D4200E583C2E3F58363A20180EA75A20022E063
:103D5200A363A201F0A3E583C2E3F58363A201DFBB
:103D6200EE75A20022E0A363A201F0A3E583C2E400
:103D7200D2E3F58363A201DFEC75A20022E0A36324
:103D8200A201F0A3E58344F8C2E5F58363A201DF53
:103D9200EC75A20022E583C2E3F583E0A363A201EE
:103DA200F0A363A201DFEE75A20022E583C2E4D292
:0A3DB200E3F583E0A363A201F0A390
:103DBC0063A201DFEC75A20022E58344F8F583E0F1
:103DCC00A363A201F0A363A201DFEE75A20022F9A6
:103DDC0022C002C004C00612FFF0D006D004D002EC
:013DEC0022B4
:10091D000A53656E643A20000A4352432065727291
:10092D006F722120000A53796E63204572726F72C7
:10093D002120000A526563204F4B2120003C2100ED
:10094D0020000ACDE5F220E4EEF1F2EEE2E5F0ED65
:10095D00EEE920E8EDF4EEF0ECE0F6E8E820EFEE5D
:10096D00200020D2D10A0020D2C8D20A000ACAE241
:10097D00E8F220EAEEEDF40A000ACAE2E8F220ED10
:10098D00E020D2D30A000ACDE5E8E7E2E5F1F2ED89
:10099D00FBE920EFE0EAE5F2202D20000ACFF0E898
:1009AD00EDFFF220F6E8EAEBE8F7E5F1EAE8E920F9
:1009BD00EFE0EAE5F220D2D12000202D20EEF8E87C
:1009CD00E1EAE020E4EBE8EDFB210A00202D20EE2A
:1009DD00F8E8E1EAE020EDEEECE5F0E020E1EBEE09
:1009ED00EAE0210A00202D20EEEA210A00202D2028
:1009FD004F7574000ACFF0E8EDFFF220D2D120F14F
:100A0D00EE20E2F0E5ECE5EDE5EC20000ACEF2E2B9
:100A1D00E5F220EDE020E7E0EFF0EEF120D2D30A91
:100A2D00000AC4E0FE20EAEEECE0EDE4F320E8F18C
:100A3D00EFEEEBEDE8F2FC20D2D30A000AD2D32080
:100A4D00E8F1EFEEEBEDE5EDEE20F3F1EFE5F8ED8E
:100A5D00EE210A000ACEF2EFF0E0E2EAE020EFEE3E
:100A6D0020F2E0E9ECE0F3F2F3000ACEF2EFF0E071
:100A7D00E2EAE020EFE0EAE5F2E020E8E720EEF739
:100A8D00E5F0E5E4E8003E2A2C312CCFE0F0E0EC77
:100A9D00E5F2F0FB20F1E8EDF5F0EEEDEDEEE3EE35
:100AAD0020EFEEF0F2E00A003E4C2C4230312C25C6
:100ABD006C752CD1EAEEF0EEF1F2FC20EEE1ECE5F6
:100ACD00EDE02C35302C3130302C3230302C3330B1
:100ADD00302C3630302C313230302C323430302C0A
:100AED00343830300A003E422C4731302C256275A7
:100AFD002CC8EDE2E5F0F1E8FF20EDE020EFF0E8A5
:100B0D00B8ECE50A003E422C4731312C2562752C9C
:100B1D00C8EDE2E5F0F1E8FF20EDE020EFE5F0E5CE
:100B2D00E4E0F7E50A003E422C4730322C25627591
:100B3D002CD3EFF0E0E2EBE5EDE8E520EFEEF2EEA1
:100B4D00EAEEEC2020285254532D435453290A0029
:100B5D003E532C4730332C256C752CC7E0E4E5F063
:100B6D00E6EAE020F1F2E0F0F2E020EFE5F0E5E476
:100B7D00E0F7E828ECF1290A003E2A2C312CCCEEC6
:100B8D00F1F2EEE2EEE920EAEEEDF2F0EEEBEBE55E
:100B9D00F020CACF2022C8F1E5F2FC222E20CFF0A2
:100BAD00EEF2EEEAEEEB2022C3F0E0EDE8F22220C9
:100BBD002D20F1E8EDF5F0EEEDEDFBE92C2000EA4E
:100BCD00EBE0F1F1E8F7E5F1EAE8E92E0A00F0E0F3
:100BDD00F1F8E8F0E5EDEDFBE92E0A003E422C4779
:100BED0030312C2562752CD0E0F1F8E8F0E5EDED13
:100BFD00FBE920EFF0EEF2EEEAEEEB0A003E532CAD
:100C0D004730342C2562752CCDEEECE5F020CACFA3
:100C1D000A003E432C4731392C25732CCAEEEDF4D6
:100C2D00E8E3F3F0E0F6E8FF20CACF3A0A0020250A
:100C3D0062752020202562752020202025627520D8
:100C4D00202025627520003E532C4731382C25730A
:100C5D002CF1F2E0F0F2EEE2FBE520EDEEECE5F04A
:100C6D00E020C0D4C13A0A003E422C4730352C2535
:100C7D0062752CCCE0E3E8F1F2F0E0EBFCEDFBE982
:100C8D0020F0E5E6E8EC0A003E422C4730362C25F4
:100C9D0062752CD2D120EFEE20E7E0EFF0EEF1F30C
:100CAD000A003E422C4730372C2562752CD2C8D213
:100CBD0020EFEE20E7E0EFF0EEF1F30A003E532CCB
:100CCD004730382C2562752CD2E0E9ECE0F3F220A8
:100CDD00EFE5F0E5F5EEE4E020EA20E8EDE8F6E8F2
:100CED00E0F2E8E2EDEEE920EFE5F0E5E4E0F7E52E
:100CFD002863290A003E4C2C4730392C256C752C65
:100D0D00CAEEEDF42E20D2D32C3136202D20EFF06B
:100D1D00FFECEEE520F3EFF02E2C3330202D20F1FB
:100D2D0020E8F1EF2E20F0E5EBE52C313238202DC7
:100D3D0020C1D0CF20C3F0E0EDE8F20A003E422CF6
:100D4D004731342C2562752C2B20ECE5E0EDE4F0D9
:100D5D0020EFE5F0E5E420EEF2EAF0FBE2E0FEF94B
:100D6D00E8EC20F4EBE0E3EEEC0A003E422C4732D7
:100D7D00312C2562752CC1EBEEEAE8F0EEE2E0F2E3
:100D8D00FC20D2D120F120ECE5F2EAE0ECE820E203
:100D9D00F0E5ECE5EDE80A003E422C4731352C2517
:100DAD0062752CCFE5F0E5E4E0E2E0F2FC20E0F046
:100DBD00F5E8E220D2D120EFF0E820F1F2E0F0F2F8
:100DCD00E50A003E422C4732352C2562752CD2C8DF
:100DDD00D220EAE0EA20E220D1E8F1F2E5EB0A00C8
:100DED003E532C4731372C25732CD0E5E2E5F0F13D
:100DFD00E8E2EDFBE520D2C8D20A003C4230313D9D
:100E0D00003C4731303D003C4731313D003C4730DF
:100E1D00323D003C4730333D003C4730313D003CD6
:100E2D004730343D003C4730353D003C4730363D82
:100E3D00003C4730373D003C4730383D003C4730A3
:100E4D00393D003C4731353D003C4732353D003C96
:100E5D004731343D003C4732313D003C4731373D51
:100E6D00000008040C020A060E0109050D030B070C
:100E7D000F00112332465765748C9DAFBECADBE956
:100E8D00F810013322564775649C8DBFAEDACBF94D
:100E9D00E82130021367764455ADBC8E9FEBFAC83E
:100EAD00D93120120377665445BDAC9E8FFBEAD82D
:100EBD00C94253617004152736CEDFEDFC8899AB1E
:100ECD00BA5243716014053726DECFFDEC9889BB0D
:100EDD00AA6372405125340617EFFECCDDA9B88AFE
:100EED009B7362504135241607FFEEDCCDB9A89AED
:100EFD008B8495A7B6C2D3E1F008192B3A4E5F6DDE
:100F0D007C9485B7A6D2C3F1E018093B2A5E4F7DCC
:100F1D006CA5B48697E3F2C0D129380A1B6F7E4CBD
:100F2D005DB5A49687F3E2D0C139281A0B7F6E5CAC
:100F3D004DC6D7E5F48091A3B24A5B69780C1D2F9D
:100F4D003ED6C7F5E49081B3A25A4B79681C0D3F8C
:100F5D002EE7F6C4D5A1B082936B7A48592D3C0E7D
:100F6D001FF7E6D4C5B1A092837B6A58493D2C1E6C
:100F7D000F0089129B24AD36BF48C15AD36CE57E54
:100F8D00F78108931AA52CB73EC940DB52ED64FFDB
:100F9D0076028B109926AF34BD4AC358D16EE77CCB
:100FAD00F5830A9118A72EB53CCB42D950EF66FDBB
:100FBD0074048D169F20A932BB4CC55ED768E17AAB
:100FCD00F3850C971EA128B33ACD44DF56E960FB9B
:100FDD0072068F149D22AB30B94EC75CD56AE3788B
:100FED00F1870E951CA32AB138CF46DD54EB62F97B
:100FFD007008811A932CA53EB740C952DB64ED767B
:10100D00FF89009B12AD24BF36C148D35AE56CF75A
:10101D007E0A8318912EA73CB542CB50D966EF744A
:10102D00FD8B029910AF26BD34C34AD158E76EF53A
:10103D007C0C851E9728A13AB344CD56DF60E9722A
:10104D00FB8D049F16A920BB32C54CD75EE168F31A
:10105D007A0E871C952AA338B146CF54DD62EB700A
:10106D00F98F069D14AB22B930C74ED55CE36AF1FA
:0F107D0078D2D120D2C8D220D2D320D2C8C80076
:105C110052600000000000000000000000000000D1
:105C210000000000004A646900000000000000005C
:025C3100000071
:105CC500906FBFE06FFC900F7E93FE906FBCE06E0F
:0F5CD500906FBFF0AF04EF900E7E93906FBCF016
:015CE400229D
:10001E00EF540F900E6E93FEC454F0FEEFC4540FC7
:04002E00932EFF22EC
:105BA90030202CE4907D51F0E57C24FEFFA3F09099
:105BB9007F56E0907D53F0A37408F0906E3D63A288
:105BC90001907D5563A201123CDFC2207F01227F33
:025BD9000022A8
:10591B00C232E4FEE57A64056032BF7E07D206E44C
:10592B00F575F57AEF30E707436B01057A8006537F
:10593B006BFEE4F57A0575E575B40808856B7FD2C7
:10594B0032E4F575E56B25E0F56B800CEF30E70580
:10595B00D206A23222E4F57AEF25E0FF0EBE08B4A0
:02596B00A23266
:01596D002217
:10568D00E4FEE57425E0F574EF30E7364374012050
:10569D0033330573E573B4052CE4F5730579E579BA
:1056AD00B408170571E571AC707002057014F582C0
:1056BD008C83E574F0057DE4F579E57425E0F574EA
:1056CD008003E4F5730579E579B408170571E57183
:1056DD00AC707002057014F5828C83E574F0057D55
:0D56ED00E4F579EF25E0FF0EEE64087095FE
:0156FA00228D
:0447A9008E338F3488
:1047AD00906FBCE0907F6EF0906FBFE0907F6FF0E8
:1047BD00E4F57DF573906FBCF0906FBFF0AB34AA4C
:1047CD003375706E7571CD3014258571828570834A
:1047DD00740AF00571E57170020570F582857083BC
:1047ED0074AAF00571E57170020570057D057D8572
:1047FD007182857083747EF00571E57170020570AC
:10480D00057DE4F579907F6CF0907F6CE0C39D5051
:10481D004B8B828A83E0FF12001E907F6DEFF0902C
:10482D006FBFE06F907F6DF0E0FF900F7E93FE9075
:10483D006FBCE06E906FBFF0EF900E7E93906FBCEB
:10484D00F00BEBAE0270010A14F5828E83E0FFC20D
:10485D003312568D907F6CE004F080AD906FBFE009
:10486D00FF12001EC23312568D906FBCE0FF120076
:10487D001EC23312568DD2337F7E12568DD233E443
:10488D00FF12568DD2037C6E7DCD8C708D71302FC5
:10489D00097E097F1DAB7D1249BC907F6EE0906F44
:0A48AD00BCF0907F6FE0906FBFF049
:0148B70022DE
:0100320022AB
:104EE900E4FF0F24E0F582E43479F5837408F00FC8
:104EF90074E02401F582E43479F583E4F07C607D83
:104F090005FEED1DAA0470011CF5828A83E0FBAA47
:104F1900070F74E02AF582E43479F583EBF00EBECD
:104F290004E07C607D09E4FEED1DAA0470011CF516
:104F3900828A83E0FBAA070F74E02AF582E43479B8
:104F4900F583EBF00EBE04E07C607D0DE4FEED1D03
:104F5900AA0470011CF5828A83E0FBAA070F74E09A
:104F69002AF582E43479F583EBF00EBE04E07C6027
:104F79007D11E4FEED1DAA0470011CF5828A83E00F
:104F8900FBAA070F74E02AF582E43479F583EBF084
:044F99000EBE04E064
:014F9D0022F1
:105D3C00D291D209E4F57CF57A906FBFF0906FBCEC
:0A5D4C00F0F575756D6E756E3D2261
:10455600200903024650E56554386560700302463B
:1045660087E56024085438F560131313541F24504C
:10457600F8E6F57820063020082DFF12591B50D694
:10458600AF7F12001E125CC5056EE56EAE6D700241
:10459600056D14F5828E83E57FF0057CE57CD3946A
:1045A6004040B3D20880AFE57CD394024005200892
:1045B60002D220C209C206E4F54ED23BC291906FE8
:1045C600BFE0FF906FBCE04F6037C220302F0D7EFA
:1045D600097F257C6E7D3DAB7C1249BC90600A123A
:1045E6002CB8E47B01FAF9F8122B6F90600A122CB2
:1045F600D0906E3DE0704E20084BC23B125D3C8071
:1046060044906E3DE07014C220302F397E097F320F
:104616007C6E7D3DAB7C1249BC802A302F0D7E0915
:104626007F407C6E7D3DAB7C1249BC906002122CB3
:10463600B8E47B01FAF9F8122B6F906002122CD0C5
:10464600E49078C1F0C20802455C203B34E550B4E2
:104656007E0F300408E4F54ED23BC20422125D3CC4
:1046660022E550B56716200713D20190601CE0FFC3
:10467600A3E09065F8CFF0A3EFF0C20AE4F54ED2BE
:024686003B22D5
:0B5DC300301F05C21F7F01227F00225D
:104F9E009078D974FFF0A374B8F0E49078D8F090BC
:104FAE0078C504F09064737410F0C207C20FC20D7E
:104FBE00D20BC20CC21190601C7402F0A374EEF0FE
:104FCE001234B5300B07906F7AE0B4010E90601A70
:104FDE007410F09060177402F0800C90601A7408D0
:104FEE00F09060177404F0E4906051F0906018F047
:104FFE00C215C21AC216C217D21ED21D906FBEF0B3
:10500E00907F6BF0907F6BE0FFC394085018EF25F4
:10501E00E024BDF582E4346EF583E4F0A3F0907FD6
:10502E006BE004F080DE9078C37402F0A37471F02C
:10503E0090601CE0FFA3E09065F8CFF0A3EFF012B4
:02504E0056FB0F
:01505000223D
:015DCE0022B2
:102DC200756A7E3007047F5580027FA08F67C20933
:102DD200D213C220D23BC21CC203C21FD201C217ED
:102DE200E4906E3CF09078C6F0907F6BF0907F6B31
:102DF200E0FFC3947F501475F009EF906FC0122D5D
:102E02000DE4F0907F6BE004F080E2E4906016F055
:102E1200906F4D7464F0E49065FAF0A3F090601244
:102E2200F0A3F0A3F0A3F0906F7BF090601BF07B17
:102E3200017A6F797C906474122D227A617968909C
:102E4200604E122D22E4907F74F0A3F0A3F0A3044D
:102E5200F0907F76E0FCA3E0FDC39405EC94004083
:102E620003022EE5907F75E0C4F8540FC868FF9006
:102E72007F74E0C454F0487E00EF5430FFED2FFF22
:102E8200EE3C907F70F0A3EFF0E4907F6EF0A3F041
:102E9200907F71E0FF906474122D19EF1229EB906C
:102EA2006474122D19900001E41229FD906475E4F6
:102EB20075F002122AAA907F6EE475F001122AAA16
:102EC200907F6EE07004A3E0640870C4907F76E4A3
:102ED20075F001122AAA907F74E475F001122AAAF1
:102EE200022E53E4907F6BF07E097F4A125329EF42
:102EF2004E7021907F6BE0FF90780093FE74522F0A
:102F0200F582E43460F583EEF0907F6BE004F0E04C
:102F120070E18019907F6BE02452F582E43460F511
:102F2200837401F0907F6BE004F0E070E7E4907F3F
:102F32006DF0907F6CF0907F6BF0907F6BE0247768
:102F4200F582E43464F583E0FF7003023034907F4D
:102F52006CE0C3748094814003023034EFB42008E3
:102F6200907F6BE004F080D2907F6BE02477F58253
:102F7200E43464F583E0642D7037907F6BE004F0F5
:102F8200E02477F9E43464FA7B01C0031B8B3175CA
:102F92003200753300E4F534D003123DED907F6DBD
:102FA200EFF0907F6CE0FEC3EF9EA3F0E004F080B0
:102FB20029907F6BE02477F9E43464FA7B01C00343
:102FC2001B8B31753200753300E4F534D003123DAA
:102FD200ED907F6CEFF0A37401F0907F6DE0D394DD
:102FE200004023907F6CE0FF7480948150187451EC
:102FF2002FF582E43460F583E4F0907F6CE004F016
:10300200A3E014F080D4907F6BE02477F582E4345F
:1030120064F583E0FF64207003022F3CEF642D709F
:1030220003022F3CEF7003022F3C907F6BE004F011
:1030320080D4E4907F6BF0907F72F0A3F0907F7663
:10304200F0A37405F0E4907F74F0A3F0906017E0B1
:10305200FFC3907F75E09F907F74E094004003026D
:103062003138907F73E0C4F8540FC868FF907F72C4
:10307200E0C454F0485401FEEF54F0FF907F77E033
:103082002FFF907F76E03E907F70F0A3EFF0E49008
:103092007F6EF0A3F090601AE0FFC3907F6FE09F15
:1030A200907F6EE094005077200B3A907F6BE0FFA8
:1030B20004F074522FF582E43460F583E0701090CE
:1030C2007F71E02400FF907F70E03420FE80089042
:1030D2007F70E0FEA3E0FF90604E122D19EE8FF09C
:1030E200122B238014907F70E0FEA3E0FF90604ECD
:1030F200122D19EE8FF0122B2390604E122D199083
:103102000002E4F5F0122B4290604FE475F00412D5
:103112002AAA907F6EE475F001122AAA02309790D3
:103122007F74E475F001122AAA907F72E475F001AF
:10313200122AAA02304E907F76E475F001122AAA72
:10314200907F76E07004A3E0640B6003023047C214
:0631520091C290125ACC5C
:013158002254
:105D1F00907E557444F0A37418F0A3EDF0A3EFF048
:0D5D2F00A37401F0E4A3F07F06125051228E
:1044070075F008EF90663C122D0DAF8285832E8FD5
:104417002FA3A3A3E0FF852F82852E83A3A3E02FDD
:10442700FFE433FEE52F2404F582E4352EF583E01F
:104437007C002FFFEC3EFEE52F2405F582E4352EA8
:10444700F583E02FFFEC3E4F7002FF229078C5E026
:10445700906F4EF0906FBEE024F0906F4FF0906F2A
:10446700BEE004F0540FF0906F507406F0A37491FF
:10447700F0906014E0FEA3E0906F52F0EEA3F030EE
:104487002F0D7E097F4D7C607D147B021249BC8510
:104497002F82852E83A3A3E0906F54F0852F82850A
:1044A7002E83A3A3A3E0906F55F0E52F2404F58294
:1044B700E4352EF583E0906F56F0E52F2405F5825D
:1044C700E4352EF583E0906F57F0852F82852E8394
:1044D700A3E0FB540FFEC454F0FE852F82852E8384
:1044E700E0FDC313042E906F58F0ED5403FF25E051
:1044F700FFEB5410FEC4540F2FA3F0E52F2407F54C
:1045070082E4352EF583E0FEE52F2406F582E435B7
:104517002EF583E07C002400FFEC3EFE7D0A122A84
:104527001FEF547F906F5AF0852F82852E83A3E06B
:1045370030E709906F5AE04480F08007906F5AE0A7
:0E454700547FF07E6F7F4E7D0D1247A97F01DD
:014555002243
:024E2200AB07DC
:104E240075F009EF906FC0122D0DAD82AC83E05484
:104E3400BFF00DBD00010C9078C5E0906F4EF0906E
:104E44006FBEE024F0906F4FF0906FBEE004F0541A
:104E54000FF0906F507403F0A37491F0EBC4540FEF
:104E6400240CA3F0EB540FA3F08D828C83E0906F9D
:104E740059F00DBD00010C8D828C83E0906F5AF0C7
:104E84000DBD00010C8D828C83E0906F5BF00DBD35
:104E940000010C8D828C83E0906F5CF00DBD0001ED
:104EA4000C8D828C83E0906F54F00DBD00010C8D4D
:104EB400828C83E0906F55F00DBD00010C8D828CC7
:104EC40083E0906F56F00DBD00010CAE04AF058F6A
:104ED400828E83E0906F57F0E4A3F07E6F7F4E7D67
:044EE4000F1247A9B9
:014EE80022A7
:10596E008F2E9078C5E0906F4EF0E52E24A0A3F018
:10597E00E4A3F0A37402F07E6F7F4E7D041247A95C
:10598E00302F277E097F4FE4FBFDFC1249BCE52E2C
:10599E00B4080C7E097F6FE4FBFDFC1249BC227E2D
:0B59AE00097F74E4FBFDFC1249BC22E1
:105BDB009078C5E0906F4EF0E57B24F0A3F0A374B2
:105BEB00FEF0A3748FF07E6F7F4E7D041247A9C227
:105BFB000E302F0B7E097F7AE4FBFDFC1249BC2291
:105A02009078C5E0906F4EF0907F6B740BF09064CD
:105A1200F7E0D394074006907F6BE004F0907F6B31
:105A2200E02480906F4FF0E4A3F0A3F07E6F7F4EEE
:105A32007D041247A9C202302F0B7E097F86E4FB48
:055A4200FDFC1249BC4F
:015A4700223C
:105D6C009078C5E0906F4EF0A37490F07E6F7F4EEC
:065D7C007D021247A9227E
:105C3400300A099065F8E4F0A37414F0906ECD7402
:105C4400AAF0A374A0F0E4A3F0D20375706E75718A
:055C5400CD757D032267
:10518A00E4907F6BF09078C5E0906F4EF0906FBE20
:10519A00E024F0906F4FF0906FBEE004F0540FF0EF
:1051AA00E4906F50F0A37490F0A37408F0E4A3F0B5
:1051BA00906F79E0906F54F0906F78E0906F55F0AF
:1051CA00906F77E0906F56F0906F76E0906F57F09F
:1051DA00C37464956CA3F0907F6B740BF0907F6B33
:1051EA00E0FFC3940F5014744E2FF582E4346FF528
:1051FA0083E4F0907F6BE004F080E27E6F7F4E7D67
:0E520A000F1247A99078C37407F0A37453F0F5
:015218002273
:02176100AB07D4
:10176300301E0B9078C3E4F0A37414F0C21E90787B
:10177300DFE024BE7003021D8E24FE601B24FC7078
:1017830003021C4C8000202F03021E237E097F933B
:101793007C787DDF1249BC229078E0E054E324DFBB
:1017A300700302197224A170030219F32460600309
:1017B300021E239078E2E06003021E239078E9E0A2
:1017C300FE9078E8E07C002400FFEC3E907F6BF015
:1017D300A3EFF0302F0D7E097FA97C7F7D6B7B0209
:1017E3001249BC9078E3E064066012202F03021EC6
:1017F300237E097FC7E4FBFDFC1249BC229078E1FC
:10180300E0D394074012202F03021E237E097FD9C1
:10181300E4FBFDFC1249BC229078E1E0FE54079002
:101823007F6DF0EE25E025E0F52975F002A4247C18
:10183300F9746F35F0FA7B01906474122D22E4F58C
:101843002A906474122D199000011229BEFF120010
:101853001E74E4252AF582E43478F583E06F601082
:10186300906474122D191229A544401229EBD21643
:10187300906474122D191229A544801229EB9064E7
:1018830074122D191229A5540F24C7F582E4347854
:10189300F58374C8F074E4252AF582E43478F5837B
:1018A300E0FF12001E906474122D19900001EF12D4
:1018B30029FD906475E475F002122AAA052AE52A27
:1018C300C394045003021844907F6DE025E024BDC7
:1018D300F582E4346EF583E0FEA3E0FF907F6BE0D6
:1018E300FCA3E0FDEF6D7002EE6C6071C3EF9DEE43
:1018F3009C505030004D300B4AC3ED9FFFEC9EFED1
:10190300D3EF941EEE9400501EA3E0FD25E024BD0A
:10191300F582E4346EF583E0FEA3E024FFFFEE34AA
:10192300FFFE125D1F8036907F6BE0FEA3E0FFA3F6
:10193300E025E024BDF582E4346EF583EEF0A3EFF9
:10194300F0801A907F6BE0FEA3E0FFA3E025E02484
:10195300BDF582E4346EF583EEF0A3EFF0202F03A0
:10196300021E237E097FF2E4FBFDFC1249BC229098
:1019730078E1E0FFB56F09A3E065727003021E23EF
:101983009078E3E064086003021E238F6F9078E28F
:10199300E0F572EF75F002A4240BFFE435F0FED3FB
:1019A300EF940FEE64809480400C7E097FFAE4FB91
:1019B300FDFC1249BC229078E2E014FF9078E1E04C
:1019C300C43354E02FF52975F009906FC0122D0D23
:1019D300E04440F0D2159078E463A20175F009E584
:1019E30029906FC1122D0D63A2017F08123CDF22E3
:1019F3009078E3E064086003021E239078E1E0FF3F
:101A0300D394074003021E23EF5407FF907F6DF02A
:101A1300FD9078EBE0FE9078EAE07A002400FFEA9C
:101A23003EFE907F6BF0A3EFF0ED25E024BDF58241
:101A3300E4346EF583E0FCA3E0FD2401FBE43CFA0F
:101A4300EB6F7002EA6E7003021AE8907F6BE0FAA4
:101A5300A3E0FBC3ED9BEC9A504A300B47A3E02570
:101A6300E024BDF582E4346EF583E0FEA3E0FFC31A
:101A7300EB9FFDEA9EFCD3ED941EEC94005009907D
:101A83007F6DE0FD125D1F22907F6BE0FEA3E0FF00
:101A9300A3E025E024BDF582E4346EF583EEF0A3E4
:101AA300EFF08041907F6DE0FF25E024BDF582E4F7
:101AB300346EF583E0FCA3E0FD907F6BE0FAA3E0D6
:101AC300FBC3ED9BFDEC9AFCD3ED941EEC9400500C
:101AD30003021E23EF25E024BDF582E4346EF58373
:101AE300EAF0A3EBF0302F0D7E0A7F017C7F7D6B44
:101AF3007B021249BC907F6DE025E024BDF582E4B2
:101B0300346EF583E475F001122AAA9078E2E0546A
:101B13007FFF131313541FFF9078E1E025E025E0C6
:101B23002FF52975F002A4247CF9746F35F0FA7B44
:101B330001906474122D229078E2E05407F5297520
:101B43002A806010E529D394004009E52A13F52A79
:101B5300152980F09078E2E030E717906474122D35
:101B630019E92401F9E43AFA1229A5452A1229EBC5
:101B73008018906474122D19E92401F9E43AFA12D9
:101B830029A5FFE52AF45F1229EB906474122D193D
:101B93001229A5FF540F24C7F582E43478F5837422
:101BA300C8F0EF44C01229EB300B03301B03D216ED
:101BB3002290601BE075F00890663C122D0DAF82F9
:101BC300AE839078E1E08F828E83F00FBF00010E29
:101BD3009078E2E08F828E83F00FBF00010E907841
:101BE300E4E08F828E83F00FBF00010E9078E5E072
:101BF3008F828E83F00FBF00010E9078E6E08F8214
:101C03008E83F00FBF00010E9078E7E08F828E8302
:101C1300F00FBF00010E9078E8E08F828E83F00F03
:101C2300BF00010E9078E9E08F828E83F090601BF5
:101C3300E004F0301703021E23E49065FAF0A3F0EA
:101C4300D217906FBD7403F0229078E2E0FF30E684
:101C530003021E239078E1E0FEC394064003021EB4
:101C630023752D78752EE4EF547FFFEEC43354E0D3
:101C73002FF52975F004A42468F9746135F0FA7B13
:101C83000190604E122D229078E3E0FFC313F529F3
:101C9300E4F52AE52AC395294003021E23200B7B82
:101CA300852E82852D83E0752B00F52CA3E0FEE4C1
:101CB300252CF52CEE352BF52B90604E122D191299
:101CC3002AC0E5F030E535C3E52C9478E52B648034
:101CD300946C5006752BEC752C78E52C2488FFE565
:101CE3002B3413FE7C007D28122A7490604E122D33
:101CF30019900002EE8FF0122B428039AF2CAE2BDD
:101D0300125D967C007D14122A7490604E122D1978
:101D1300900002EE8FF0122B42801A852E82852DC1
:101D230083E0FEA3E0FF90604E122D19900002EEB7
:101D33008FF0122B427402252EF52EE4352DF52D4E
:101D4300200F1390604E122D19122AC0FFE5F044A4
:101D5300408FF0122B23D21A90604E122D19122AA3
:101D6300C0FFAEF07C00540F24C7F582EC3478F545
:101D73008374C8F0EE44808FF0122B2390604FE4FD
:101D830075F004122AAA052A021C969078E2E064F0
:101D93000370659078C6E0605F302F0B7E0A7F1971
:101DA300E4FBFDFC1249BC9064F7E0FF9078E1E0AE
:101DB3006F70409078C2E0FF9078E4E06F703490E9
:101DC3007E557402F0A37408F09064F7E0907E5798
:101DD300F0A3F0A37401F0E4A3F07F061250519036
:101DE3006E3C7420F0302F0B7E0A7F2EE4FBFDFC4B
:101DF3001249BCE49078C6F09078E2E06401702068
:101E0300906E3CE0601A9078E5E07002D202E490B4
:101E13006E3CF0302F0A7E0A7F49FBFDFC1249BC61
:011E2300229C
:105B3D00906016E0FFC3947F502575F009EF906FCC
:105B4D00C0122D0DE030E60F906016E0124E22903F
:105B5D006016E004F0D322906016E004F080D1E4EA
:085B6D00906016F0C215C3227E
:10468800906F4DE06002C322C232906051E0FF603B
:1046980002D2328F2EE52EC39420400302479EE5B6
:1046A8002E131313541FF52FE52E75F002A4247C46
:1046B800F9746F35F0FA7B01906474122D22122977
:1046C800A520E603024799E52E5407FFC3E52E9F70
:1046D800F52E2408906051F0E52E75F002A4247C94
:1046E800F9746F35F0FA906474122D227E607F1E83
:1046F8009078C5E08F828E83F00FBF00010E1229DB
:10470800A5FD540F24408F828E83F00FBF00010E49
:10471800EDC4540324208F828E83F00FBF00010E56
:10472800E4F52E906474122D199000011229BE8FA1
:10473800828E83F01229A554BF1229EB74082FFF2B
:10474800E43EFE906474122D199000011229BEF403
:104758008F828E83F074F82FFF74FF3EFE9064758D
:10476800E475F002122AAA0FBF00010E052EE52EED
:10477800B408B07E607F1E7D131247A9E52F25E09F
:104788002469F582E43464F583E4F0A3747DF0D3FE
:1047980022052E02469DE4906051F0A2329216C383
:0147A80022EE
:10377000906017E0FF90601AE08FF0A475F006A447
:10378000F532906018E0F530E530C3953240030221
:1037900039ED90601AE0FFE5308FF084F531E530C7
:1037A00075F004A42468F9746135F0FA7B01906027
:1037B0004E122D22122AC0E5F020E6030239E890CD
:1037C000601AE0FFE5308FF084C3E53095F0F53006
:1037D0002F906018F0E53075F004A42468F9746146
:1037E00035F0FA90604E122D22906F7AE0B4010607
:1037F0007E607F1E80047E607F1F8E2E8F2F9078CC
:10380000C5E0852F82852E83F0052FE52F700205F8
:103810002E300B030238A590604E122D19122AC0CB
:10382000FFAEF0540F2440852F82852E83F0052FA4
:10383000E52F7002052EEEC4F854F0C868EFC454AA
:103840000F48541F2460852F82852E83F0052FE5B5
:103850002F7002052EE4F53090601AE0FFE530C3CA
:103860009F503690604E122D19900002122AEB855F
:103870002F82852E83F0122AC0FFE5F054BF8FF00F
:10388000122B2390604FE475F004122AAA052FE54D
:103890002F7002052E053080BF7E607F1F7D1312C2
:1038A00047A90239E6906F7AE064017045852F825E
:1038B000852E837470F0052FE52F7002052EF5829A
:1038C000852E837442F0052FE52F7002052E90603F
:1038D0004E122D19122AC0FFE5F0C4F854F0C86842
:1038E000EFC4540F48540F2460852F82852E83F037
:1038F0008071906FBEE024F0852F82852E83F0903A
:103900006FBEE004F0540FF0052FE52F7002052E76
:10391000F582852E837402F0052FE52F7002052EA7
:10392000F582852E837491F0052FE52F7002052E08
:1039300090604E122D19122AC0FDACF0ECC4F85460
:10394000F0C868EDC4540F48540FFBEDC4F8540F91
:10395000C868FFECC454F048EF54F02B852F8285E3
:103960002E83F0906F7AE0B401067E607F2280049F
:103970007E607F24E4F53090601AE0FDE530C39D61
:10398000503990604E122D19900002122AEBFD8FD3
:10399000828E83E5F0F0A3EDF0122AC0FDE5F0542D
:1039A000BF8DF0122B2390604FE475F004122AAA09
:1039B00074022FFFE43EFE053080BC906F7AE0FF7A
:1039C000B401067C607D1E80047C607D1F8C2E8D82
:1039D0002FEFB401047F2480027F158F30AD30AF0C
:1039E0002FAE2E1247A9D3220530023788E490600B
:0539F00018F0C21AC32B
:0139F50022AF
:1058C400D218906F4DE0704EE4F52EE52EC394206F
:1058D4005035E52E75F002A4247CF9746F35F0FA86
:1058E4007B01906474122D221229A5FF30E71090D9
:1058F4006474122D19EF44401229EBD216C21874A5
:1059040004252EF52E80C430180C906F76122CDCF2
:0659140000000000D21E9D
:01591A00226A
:105A8C00906F7BE075F00890663E122D0DAF82AEE4
:105A9C0083E4F00FBF00010E8F828E83E4F00FBF02
:105AAC0000010E8F828E83E4F00FBF00010E8F82F7
:0F5ABC008E83E4F00FBF00010E906F7BE004F0CB
:015ACB0022B8
:10108C0030122DC3E54D9569FFE54C9568FED3EF05
:10109C009440EE940040197B087D40AF69AE681215
:1010AC004C7CE5692440FFE43568540FF5688F6982
:1010BC00301D05122DC2C21D1245562022030211ED
:1010CC00C6C222906F4DE0600214F0E4F52974C79B
:1010DC002529F582E43478F583E070030211BB74A2
:1010EC00C72529F582E43478F583E014F074C7251C
:1010FC0029F582E43478F583E060030211BBE5291D
:10110C00D39404503FE52975F010A4246CF9746F46
:10111C0035F0FA7B01906474122D22E4F52AE52A4D
:10112C00C3940840030211BB906474122D19122948
:10113C00A5547F1229EB052A906475E475F0021210
:10114C002AAA80DAE52924FBFF90601AE0FEEF8ED4
:10115C00F0A4FF906017E0FEEF8EF0A475F004A4ED
:10116C002468F9746135F0FA7B0190604E122D22DF
:10117C00E4F52A906017E0FF90601AE08FF0A4FF6E
:10118C00C3E52A9FE5F06480F87480985021906044
:10119C004E122D19122AC0FFE5F0547F8FF0122B3E
:1011AC0023052A90604FE475F004122AAA80C40526
:1011BC0029E529641060030210DA20300302129B27
:1011CC00C2309078C6E0600214F0906E3CE0600291
:1011DC0014F09078C3E07002A3E0600A9078C374B6
:1011EC00FFF5F0122AAA9065FAE07002A3E0600AFB
:1011FC009065FA74FFF5F0122AAA9065F8E0700277
:10120C00A3E060349065F874FFF5F0122AAA90659B
:10121C00F8E07002A3E07020200702D201200A0837
:10122C00E49078D7F01258C4D20A302F0B7E0A7F84
:10123C0061E4FBFDFC1249BCE4F529E52925E02419
:10124C0069F582E43464F583E0FEA3E04E6037E593
:10125C002925E02469F582E43464F58374FFF5F004
:10126C00122AAAE52925E02469F582E43464F58381
:10127C00E0FEA3E04E700F300A0C200D099078D7D9
:10128C007402F01258C40529E529C3940440AC300B
:10129C002425C224906468E0600214F0D56C1875A3
:1012AC006C64906F76122CB8E47B01FAF9F8122B6F
:1012BC006F906F76122CD02020030215BCC22090A8
:1012CC0078C5E0FF906E3DE06F60030215B1A3E0BE
:1012DC00FF54F024F0603624E0700302148B244099
:1012EC0070030214A424F060030215BCEF540FF534
:1012FC002BD3940440030215BCE52B25E02467F5A1
:10130C0082E43464F583E4F0A3F00215BC906E3EE5
:10131C00E0540F14607614607324F96012046003B7
:10132C000215BC9078D77401F01258C40215BCD2C7
:10133C0010906017E0FF90601AE08FF0A475F00633
:10134C00A4F52AE4F529E529C3952A40030215BC26
:10135C00E52975F004A42468F9746135F0FA7B0171
:10136C0090604E122D22122AC0FFAEF0EE30E71222
:10137C0090604E122D19EE44408FF0122B23D21A8E
:10138C00C21090601AE02529F52980BA9078C6E041
:10139C0060030215BC906E3CE060030215BC906EBD
:1013AC0044E0F4FF906E3FE0FE6F60030215BC90CA
:1013BC006E45E0F4FF906E40E0FD6F60030215BCDB
:1013CC00906E46E0F4FF906E41E06F60030215BC36
:1013DC00E4F5298E2BED6009752908906E40E0F537
:1013EC002BE4F52AE52B20E70F0529E52B25E0F565
:1013FC002B052AE52AB408EC906473E0FF13131351
:10140C00541FFFE5298FF0849064F7F0E5298FF0E5
:10141C008485F029E52933333354F8F529906E414E
:10142C00E0F52BE4F52AE52B20E70F0529E52B2524
:10143C00E0F52B052AE52AB408ECE52925E090789F
:10144C00C2F0906E3EE020E0079078C2E04401F0DC
:10145C00907E557442F0A37418F09064F7E0907E7F
:10146C0057F09078C2E0907E58F0A37401F0E4A39A
:10147C00F07F061250519078C6740AF00215BC30F9
:10148C000702D20190601CE0FFA3E09065F8CFF05A
:10149C00A3EFF0C20A0215BC906E40E024C0606558
:1014AC0024FE607924F360030215BC906E3FE0705B
:1014BC00030215BC906E42E0FE906E41E07C00246D
:1014CC0000F52DEC3EF52C906014E0652C7004A317
:1014DC00E0652D60030215BC302F0D7E097F4D7C1D
:1014EC00607D147B021249BC906014E475F001120B
:1014FC002AAA125A8C906FBD7403F0E49065FAF02E
:10150C00A3F00215BC906E3FE0648060030215BC32
:10151C00D20E906E3EE0540FF57B0215BC906E3FE0
:10152C00E060030215BC906E41E0906F79F0906E14
:10153C0042E0906F78F0906E43E0906F77F0906E91
:10154C0044E0906F76F0906E45E0FFC374649FF5B5
:10155C006CE49078C3F0A3F0D20E906E3EE0540F82
:10156C00F57B907E557401F0A37408F0A37480F0A1
:10157C00A37401F0A37406F0906E4163A201907EF7
:10158C005A63A2017F04123CDF906E45E075F00AAD
:10159C00A485F02CF52D907E5EF0E52CA3F07F0B4E
:1015AC00125051800B906E3DE07002D204C220228A
:1015BC00301C63E56665616048E56624085438FFB5
:1015CC00E56154386F60047E0180027E00E57D6029
:1015DC00047D0180027D00EE5D70030217600571D1
:1015EC00E571AC707002057014F5828C83E0FEE539
:1015FC0066131313541F2458F8A6068F66157D80A6
:10160C00B8C21CC203D2B1300A099065F8E4F0A349
:10161C007414F0C29022300903021760A2018203F5
:10162C00505CE5666561600302176030B10AC2B1B7
:10163C00906019E0906468F030190C30B009906437
:10164C0068E060030217600571E571AE7070020509
:10165C007014F5828E83E0FFE566131313541F2478
:10166C0058F8A607E56624085438F566157DD21C93
:10167C00C201E57D64027003021760D29022200142
:10168C000302176090601BE0FE906F7BE0FF6E60C2
:10169C005C9065FAE07002A3E0705430030302170B
:1016AC0060300A04906FBDF0124407EF640170368D
:1016BC007F32125DB8302F0D7E0A7F777C6F7D7B79
:1016CC007B011249BC9065FAE4F0A37419F0906F99
:1016DC00BDE0600214F0906FBDE07078125A8C90EF
:1016EC006FBD7403F022906F7BE004F022C21730C0
:1016FC000204125A0222300E07201704125BDB225E
:10170C009078C3E07002A3E0700412518A22301862
:10171C00087F0812596EC2182220170830160512BD
:10172C00468840303010087F0912596EC2102220B2
:10173C001708301505125B3D401A301A0512377028
:10174C004012E566B5610D300704125D6C22200570
:04175C0003125C34E4
:011760002266
:1039F6009078D8E06022A3E0FEA3E0FFC3E49FFF37
:103A0600E49EFEAB07FA3395E0F9F87F007EC27DAF
:103A1600017C00125A4880219078D9E0FEA3E0FF8D
:103A2600C3E49FFFE49EFEAB07FA3395E0F9F8E4A2
:103A36007F207E1CFDFC125A488F318E308D2F8CD4
:103A46002E7BFF7A0A79931231BB7BFF7A0A79B50E
:103A5600853138853037852F36852E351231BB7B3B
:103A6600FF7A0A79F3A211E433F5351231BB7BFFF5
:103A76007A0B7912A20CE433F5351231BB7BFF7A4F
:103A86000B7933A219E433F5351231BB7BFF7A0B80
:103A9600795D906019E075F00AA4FFAEF0E48F3806
:103AA6008E37F536F5351231BB7535FF75360B7524
:103AB60037867B017A7F796B1231B5200B14753509
:103AC600FF75360B7537CC7B017A7F796B12586C94
:103AD60080127535FF75360B7537DB7B017A7F797A
:103AE6006B12586C7B017A7F796B1231BB7BFF7A44
:103AF6000B79E9A20BE433F5351231BB7BFF7A0C67
:103B0600790A9078C5E0F5351231BB7535FF753603
:103B16001075377E7BFF7A0C791F1231BB7535FF26
:103B260075360C75373B753801753905753A0B7561
:103B36003B0D7B017A6179521231B57535017536C7
:103B4600617537527BFF7A0C79541231BB7BFF7A51
:103B56000C7975A207E433F5351231BB7BFF7A0C7D
:103B66007995A20DE433F5351231BB7BFF7A0C79DA
:103B7600AFA20FE433F5351231BB90601CE0FEA313
:103B8600E0FF7C007D06122A1F8F357BFF7A0C79B9
:103B9600CA1231BB7BFF7A0D7902906473E0FFE4B1
:103BA6008F38F537F536F5351231BB7BFF7A0D794F
:103BB6004AA214E433F5351231BB300B2E7BFF7A63
:103BC6000D7978A21BE433F5351231BB7BFF7A0DF4
:103BD60079A5A200E433F5351231BB7BFF7A0D7966
:103BE600D0906F7AE0F5351231BB22753501753606
:0D3BF600647537777BFF7A0D79ED1231BBD6
:013C0300229E
:1034B5007E097F4A125329EF4E70037F01227E0E4B
:1034C5007F08125329EF4E6071125759907F6E1283
:1034D5002CD0E4FFFEFDFC907F6E122CC4C3122C91
:1034E500A76020907F6E122CC4E47F207E1CFDFC1B
:1034F500122C07122C999078D9EEF0A3EFF0E490F6
:1035050078D8F0E47FB07E04FDFC907F6E122CC469
:10351500D3122CA740339078D87401F0907F6E12A7
:103525002CC47F007EC27D017C00122C07122C99D1
:103535009078D9EEF0A3EFF0800F9078D974FFF072
:10354500A374B8F0E49078D8F07E0E7F0E1253295C
:10355500EF4E600C125D56EF24D024FF92118002CD
:10356500C2117E0E7F14125329EF4E600C125D5668
:10357500EF24D024FF920C8002C20C7E0E7F1A121B
:103585005329EF4E600C125D56EF24D024FF92199B
:103595008002C2197E0E7F20125329EF4E6013124E
:1035A5005759E47B0AFAF9F8122C07906019EFF0E5
:1035B5008005E4906019F07E0E7F26125329EF4EA8
:1035C500600C125D56EF24D024FF920B8002D20BC3
:1035D5007E0E7F2C125329EF4E600A1257599078B0
:1035E500C5EFF08005E49078C5F07E0E7F3212536A
:1035F50029EF4E600C125D56EF24D024FF92078010
:1036050002C2077E0E7F38125329EF4E600C125D01
:1036150056EF24D024FF920D8002C20D7E0E7F3E10
:10362500125329EF4E600C125D56EF24D024FF9201
:103635000F8002C20F7E0E7F44125329EF4E601693
:10364500125759E47B06FAF9F8122B7C90601CEEB0
:10365500F0A3EFF0800A90601C7402F0A374EEF002
:103665007E0E7F4A125329EF4E600A125759906415
:1036750073EFF080069064737410F07E0E7F501225
:103685005329EF4E600C125D56EF24D024FF9200B3
:103695008002C2007E0E7F56125329EF4E600C1237
:1036A5005D56EF24D0906F7AF08005E4906F7AF044
:1036B5007E0E7F5C125329EF4E600C125D56EF248F
:1036C500D024FF92148002C2147E0E7F6212532909
:1036D500EF4E600C125D56EF24D024FF921B800242
:1036E500C21B7E0E7F68125329EF4E6058E4907F0F
:1036F5006CF0125D56907F6DEFF0643C6047907FF3
:103705006DE0FF907F6CE0FE04F074772EF582E4A7
:103715003464F583EFF0125D56907F6DEFF0643CF5
:103725006009907F6CE0C3948040D3907F6CE0B4D7
:10373500800214F0907F6CE02477F582E43464F520
:1037450083E4F08023907F6CE0FF04F074772FF51D
:1037550082E43464F5837420F0907F6CE02477F57F
:0A37650082E43464F583E4F07F0091
:01376F002237
:015DCF0022B1
:105D8200BF360BD212E4F54CF54DF568F569BF3715
:045D920002C2122215
:1056FB00C2A94389029078DAE0FFF58C8F8A75D9BD
:10570B000475DA4875DB3175DC4975DD4975DE31B9
:10571B00E4F5E9F5F9F5EBF5FB9078D8E060167553
:10572B00EC1075ED10E4F5FCF5FD75640875621071
:10573B00756301801375EC8075ED80E4F5FCF5FD68
:0E574B00756480F562756310E4F5EEF5FE22DC
:105ACC00E4FEAF8CEFFD9078D9E07003A3E06D603D
:105ADC00051256FB7E01E5D920E2057E021256FB2B
:105AEC00E58920E1051256FB7E03D28C75D84075F2
:085AFC00B740D2AED2AFAF06F5
:015B0400227E
:030033000241186F
:0B411800C0E0C083C082C0D075D0089A
:10412300C2AF30DC56C3E5EC95EEC395645012E59F
:104133006325ECF5EC30D70405FC801685FCFC8088
:1041430011C3E5EC9563F5EC30D70415FC800385CA
:10415300FCFC301224854D82854C83E590F0054D9F
:10416300E54D7002054CF582854C83E5EEF0054D77
:10417300E54D7002054C534C0FC2DC30D929301287
:1041830024854D82854C83E590F0054DE54D700205
:10419300054CF582854C83E5EBF0054DE54D70024A
:1041A300054C534C0FC2D930DA6AE562700405FC42
:1041B3008010E56225ECF5EC30D70405FC8003851F
:1041C300FCFC30134DE54E5480F54BE54E25E0F5F0
:1041D3004E309702054E201103634E01303B19E523
:1041E3004E656A6006E54E65677027756000756504
:1041F30000854E50C23B801A0565E5655407701271
:1042030053653FE565131313541F2450F8A64E75E9
:104213004E00C2DA30DB71E562700405FD8010E503
:104223006225EDF5ED30D70405FD800385FDFDE541
:104233006665616029E56154077013E56113131323
:10424300541F2458F8E6F54F200C03634FFFE54F46
:10425300339296E54F25E0F54F056153613FB292E6
:10426300301223854D82854C83E590F0054DE54D55
:104273007002054CF582854C83E4F0054DE54D70E5
:0A42830002054C534C0FC2DBD2AF12
:09428D00D0D0D082D083D0E03201
:10522500021E24E493A3F8E493A34003F68001F25D
:1052350008DFF48029E493A3F85407240CC8C3338A
:10524500C4540F4420C8834004F456800146F6DF59
:10525500E4800B0102040810204080905C0BE47E82
:10526500019360BCA3FF543F30E509541FFEE4934E
:10527500A360010ECF54C025E060A840B8E493A315
:10528500FAE493A3F8E493A3C8C582C8CAC583CA40
:10529500F0A3C8C582C8CAC583CADFE9DEE780BEF8
:015C33000070
:1029A500BB010689828A83E0225002E722BBFE0230
:0929B500E32289828A83E4932263
:1029BE00BB010CE58229F582E5833AF583E02250CE
:1029CE0006E92582F8E622BBFE06E92582F8E22218
:0D29DE00E58229F582E5833AF583E4932232
:1029EB00BB010689828A83F0225002F722BBFE01CB
:0229FB00F322C5
:1029FD00F8BB010DE58229F582E5833AF583E8F010
:102A0D00225006E92582C8F622BBFE05E92582C8BB
:022A1D00F222A3
:102A1F00BC000BBE0029EF8DF084FFADF022E4CC9B
:102A2F00F875F008EF2FFFEE33FEEC33FCEE9DEC64
:102A3F00984005FCEE9DFE0FD5F0E9E4CEFD22EDAA
:102A4F00F8F5F0EE8420D21CFEADF075F008EF2FF4
:102A5F00FFED33FD4007985006D5F0F222C398FDE5
:052A6F000FD5F0EA2282
:102A7400C2D5EC30E709B2D5E4C39DFDE49CFCEE7D
:102A840030E715B2D5E4C39FFFE49EFE122A1FC3AC
:102A9400E49DFDE49CFC8003122A1F30D507C3E4A7
:062AA4009FFFE49EFE22EC
:102AAA00C5F0F8A3E028F0C5F0F8E58215827002B7
:062ABA001583E038F02254
:102AC000BB010A89828A83E0F5F0A3E022500687E1
:102AD000F009E71922BBFE07E3F5F009E3192289A3
:0B2AE000828A83E493F5F074019322D6
:102AEB00BB0110E58229F582E5833AF583E0F5F029
:102AFB00A3E0225009E92582F886F008E622BBFE06
:102B0B000AE92582F8E2F5F008E222E5832AF5834B
:082B1B00E993F5F0A3E9932210
:102B2300BB010A89828A83F0E5F0A3F0225006F7FD
:0F2B330009A7F01922BBFE06F3E5F009F31922FA
:102B4200F8BB0111E58229F582E5833AF583E8F0C5
:102B5200E5F0A3F0225009E92582C8F608A6F02282
:0D2B6200BBFE09E92582C8F2E5F008F22269
:0D2B6F00EF2BFFEE3AFEED39FDEC38FC22B5
:102B7C00E88FF0A4CC8BF0A42CFCE98EF0A42CFCF8
:102B8C008AF0EDA42CFCEA8EF0A4CDA8F08BF0A476
:102B9C002DCC3825F0FDE98FF0A42CCD35F0FCEBD5
:102BAC008EF0A4FEA9F0EB8FF0A4CFC5F02ECD399A
:0F2BBC00FEE43CFCEAA42DCE35F0FDE43CFC2207
:102BCB0075F008758200EF2FFFEE33FECD33CDCCC1
:102BDB0033CCC58233C5829BED9AEC99E582984044
:102BEB000CF582EE9BFEED9AFDEC99FC0FD5F0D621
:102BFB00E4CEFBE4CDFAE4CCF9A88222B800C1B94B
:102C0B000059BA002DEC8BF084CFCECDFCE5F0CB88
:102C1B00F97818EF2FFFEE33FEED33FDEC33FCEBC1
:102C2B0033FB10D703994004EB99FB0FD8E5E4F97C
:102C3B00FA227818EF2FFFEE33FEED33FDEC33FC69
:102C4B00C933C910D7059BE99A4007EC9BFCE99A5D
:102C5B00F90FD8E0E4C9FAE4CCFB2275F010EF2FA2
:102C6B00FFEE33FEED33FDCC33CCC833C810D707A2
:102C7B009BEC9AE899400AED9BFDEC9AFCE899F8DD
:0E2C8B000FD5F0DAE4CDFBE4CCFAE4C8F92270
:105A4800C2D5E830E70FB2D5E4C39BFBE49AFAE489
:105A580099F9E498F8EC30E717B2D5125A7E122C6F
:105A680007E4C39BFBE49AFAE499F9E498F8800305
:105A7800122C0730D50DE4C39FFFE49EFEE49DFD84
:045A8800E49CFC227C
:0E2C9900C3E49FFFE49EFEE49DFDE49CFC224C
:102CA700EB9FF5F0EA9E42F0E99D42F0E89C45F083
:012CB70022FA
:0C2CB800E0FCA3E0FDA3E0FEA3E0FF228F
:0C2CC400E0F8A3E0F9A3E0FAA3E0FB2293
:0C2CD000ECF0A3EDF0A3EEF0A3EFF02277
:102CDC00A8828583F0D083D082122CF3122CF312AD
:102CEC002CF3122CF3E473E493A3C583C5F0C583D2
:102CFC00C8C582C8F0A3C583C5F0C583C8C582C842
:012D0C0022A4
:0C2D0D00A42582F582E5F03583F58322D1
:092D1900E0FBA3E0FAA3E0F922BB
:092D2200EBF0A3EAF0A3E9F022B2
:10315900E5412435F8E605412278323039027835DF
:10316900E475F001122D2B0229A52032EB7F2ED216
:10317900328018EF540F2490D43440D4FF30360BEA
:10318900EF24BFB41A0050032461FFE54260021521
:10319900420545E5457002054430390D7832E4753C
:1031A900F001122D2BEF0229EB0259B97403D23920
:1031B9008003E4C239F5418B328A338934E4F5421C
:1031C900F544F545E54260077F2012319480F57595
:1031D90043FFC233C232C234C235C237C238C23ADF
:1031E900123162FF700D3039057F001231A5AF45EC
:1031F900AE4422B4255FC2D5C236123162FF24D053
:10320900B40A00501A75F00A784230D50508B6FF9D
:103219000106C6A426F620D5047002D23580D92429
:10322900CFB41A00EF5004C2E5D2360233A5D23327
:1032390080C6D23280C0D23480BCD2D580BAD237CF
:1032490080B47F201231942034077401B5420040C4
:10325900F1123159FF1231940231CDD23AD238806C
:1032690095123159FB123159FA123159F94A4B70F9
:103279000679767A347BFF20342EE542602A7E0077
:103289008E827583001229BE60060EEE654370F0CA
:10329900C2D5EBC0E0EAC0E0E9C0E0EE1233ECD001
:1032A900E0F9D0E0FAD0E0FB1229A5FF60AAEBC053
:1032B900E0EAC0E0E9C0E0123194D0E02401F9D09D
:1032C900E03400FAD0E0FBE5430460DCD543D98063
:1032D900877BFF7A3379E8D234809C791080027930
:1032E90008C238C23A8008D2D5790A8004790AC25C
:1032F900D5E543047002F543E4FAFDFEFF123159A6
:10330900FC7B08203313123159FD7B1030320A122D
:103319003159FE123159FF7B20EC3382D592D550B9
:1033290013C3E43032069FFFE49EFEE42033039D7D
:10333900FDE49CFCE4CBF8C233EC700CCFCECDCCD1
:10334900E824F8F870F38017C3EF33FFEE33FEED8E
:1033590033FDEC33FCEB33FB994002FB0FD8E9EB6F
:10336900303305F8D0E0C448B233C0E00AEC4D4E22
:103379004F78207B0070C2EAB5430040BCC0E01220
:1033890033EED0F0D0E0203304C4C0E0C4B233C07F
:10339900F012317DD0F0D5F0EB0231CD122D8A3209
:1033A9006A5332E458323B4C32374232E84F32F0FA
:0F33B9004432F04932504332F65532DA4632DAB6
:1033C8004532DA47349650323F2D32432E32662B3F
:1033D800324723326420347F2A31FF480000325EAE
:1033E8003F3F3F00790AA2D5203514303709B9107C
:1033F800020404B9080104A2D520380250010420AF
:1034080034689234B542005034C0E07F203035191A
:103418007F30A23472387237500F123445C234C22A
:1034280038C237C23A7F30800F303703E9C0E01224
:103438003194303703D0E0F9D0E0B542CC303717BB
:103448007F30B9100C1231947F583036077F78805E
:1034580003B908031231943034057F2D0231947F6B
:1034680020203AF87F2B2038F322923480CF286E20
:10347800756C6C2900D2331231593033F8C2337865
:103488004230D50108F60231FF2D50434958123118
:10349800592403B405004001E49034919312318516
:0D34A800743A123185D2357542040232E4C7
:105D9600C3EE6480948040028007C3E49FFFE49EC4
:025DA600FE22DB
:10586C008B328A3389348B388A39893AAB32053496
:10587C00E534AA337002053314F91229A570ED74BE
:10588C00FF2534F53474FF3533F533AB350537E587
:10589C0037AA367002053614F91229A5FFAB32056A
:1058AC0034E534AA337002053314F9EF1229EB7086
:0858BC00DAAB38AA39A93A223F
:103DED008B2E8A2F8930E4F53AF539F538F537F50C
:103DFD0035F536E532453345316012EBC0E0EAC0AA
:103E0D00E0E9C0E0AB31AA32A933122D3BAB2E0550
:103E1D0030E530AA2F7002052F14F91229A5F53BB4
:103E2D00C394094007E53BD3940D40E1E53B642085
:103E3D0060DBE53BB42D054336038016E53BB42B23
:103E4D0005433601800C74FF2530F53074FF352F96
:103E5D00F52FE53460046410703FAB2EAA2FA93006
:103E6D001229A564306009E534702E75340A802955
:103E7D009000011229BEFF64786004EFB45813431B
:103E8D00360175341074022530F530E4352FF52FD9
:103E9D008007E5347003753408AB2E0530E530AA84
:103EAD002F7002052F14F91229A5F53BC39461401B
:103EBD000AE53BD3947A5003533BDF74D0253BF591
:103ECD003BC3940A400CE53B9411406D74F9253BBE
:103EDD00F53BE53BD395345060433601853A3F853C
:103EED00393E85383D85373CAF347E00E4FCFDAB73
:103EFD003AAA39A938A837122B7CC8ECC8C9EDC924
:103F0D00CAEECACBEFCBE4FCFDFEEB253BF53AEE5A
:103F1D003AF539ED39F538EC38F537AF3AAE39AD0C
:103F2D0038FCAB3FAA3EA93DA83CD3122CA75003A9
:103F3D00023EA6433604023EA6E53620E003E480A9
:103F4D002DE53245334531601EAB2EE53024FFF9AA
:103F5D00E52F34FFFAEBC0E0EAC0E0E9C0E0AB3199
:103F6D00AA32A933122D3BE53630E20774FFFFFE6E
:103F7D00FDFC22E536AF3AAE39AD38AC3730E10352
:043F8D00022C992247
:102D2B00FAE6FB0808E6F925F0F618E6CA3AF622A9
:102D3B00BB011A89828A83D0F0D0E0F8D0E0F9D0B9
:102D4B00E0FAD0E0FBE8C0E0C0F0022D225016E91B
:102D5B00F8D083D082D0E0F9D0E0FAD0E0FBC0828B
:102D6B00C083022DB0BBFE16E9F8D083D082D0E031
:0F2D7B00F9D0E0FAD0E0FBC082C083022DB9226C
:102D8A00D083D082F8E4937012740193700DA3A3D8
:102D9A0093F8740193F5828883E4737402936860EC
:062DAA00EFA3A3A380DFEC
:092DB000EBF608EAF608E9F62248
:092DB900EBF208EAF208E9F2224B
:00000001FF
